Subject: help

From: Jeroen Baten <[email-masked]>
Date: Fri, 11 Jan 2002 22:23:57 +0100

Since a couple of days my appletalk doesn't work any more from Linux 2.4.10 
SuSE 7.3 to my G3.

I did a tcpdump and this is what happens after I get the login screen, enter 
my userid and password and click OK. Anybody an idea? Please?

22:12:36.036098 apple.i2rs.nl.49156 > server.i2rs.nl.afpovertcp: . ack 390 
win 60000 (DF)
22:12:51.874957 apple.i2rs.nl.49156 > server.i2rs.nl.afpovertcp: P 
465:481(16) ack 390 win 60000 (DF)
22:12:51.875030 server.i2rs.nl.afpovertcp > apple.i2rs.nl.49156: . ack 481 
win 5840 (DF)
22:13:05.984760 server.i2rs.nl.afpovertcp > apple.i2rs.nl.49156: P 
390:406(16) ack 481 win 5840 (DF)
22:13:06.036061 apple.i2rs.nl.49156 > server.i2rs.nl.afpovertcp: . ack 406 
win 60000 (DF)
22:13:22.874997 apple.i2rs.nl.49156 > server.i2rs.nl.afpovertcp: P 
481:497(16) ack 406 win 60000 (DF)
22:13:22.875143 server.i2rs.nl.afpovertcp > apple.i2rs.nl.49156: . ack 497 
win 5840 (DF)
22:13:35.984741 server.i2rs.nl.afpovertcp > apple.i2rs.nl.49156: P 
406:422(16) ack 497 win 5840 (DF)
22:13:36.036038 apple.i2rs.nl.49156 > server.i2rs.nl.afpovertcp: . ack 422 
win 60000 (DF)
22:13:53.874973 apple.i2rs.nl.49156 > server.i2rs.nl.afpovertcp: P 
497:513(16) ack 422 win 60000 (DF)
22:13:53.875072 server.i2rs.nl.afpovertcp > apple.i2rs.nl.49156: . ack 513 
win 5840 (DF)
22:14:05.984707 server.i2rs.nl.afpovertcp > apple.i2rs.nl.49156: P 
422:438(16) ack 513 win 5840 (DF)
22:14:06.036014 apple.i2rs.nl.49156 > server.i2rs.nl.afpovertcp: . ack 438 
win 60000 (DF)
22:14:24.875062 arp who-has server.i2rs.nl (Broadcast) tell apple.i2rs.nl
22:14:24.875089 arp reply server.i2rs.nl is-at 0:30:ab:2:7d:d5
22:14:24.875341 apple.i2rs.nl.49156 > server.i2rs.nl.afpovertcp: P 
513:529(16) ack 438 win 60000 (DF)
22:14:24.875418 server.i2rs.nl.afpovertcp > apple.i2rs.nl.49156: . ack 529 
win 5840 (DF)
22:14:29.874643 arp who-has apple.i2rs.nl tell server.i2rs.nl
22:14:29.874855 arp reply apple.i2rs.nl is-at 0:5:2:b1:e0:22
22:14:35.984843 server.i2rs.nl.afpovertcp > apple.i2rs.nl.49156: P 
438:454(16) ack 529 win 5840 (DF)
22:14:36.036146 apple.i2rs.nl.49156 > server.i2rs.nl.afpovertcp: . ack 454 
win 60000 (DF)
22:14:55.874991 apple.i2rs.nl.49156 > server.i2rs.nl.afpovertcp: P 
529:545(16) ack 454 win 60000 (DF)
22:14:55.875050 server.i2rs.nl.afpovertcp > apple.i2rs.nl.49156: . ack 545 
win 5840 (DF)
22:15:05.984769 server.i2rs.nl.afpovertcp > apple.i2rs.nl.49156: P 
454:470(16) ack 545 win 5840 (DF)
22:15:06.033429 apple.i2rs.nl.49156 > server.i2rs.nl.afpovertcp: . ack 470 
win 60000 (DF)
22:15:26.875008 apple.i2rs.nl.49156 > server.i2rs.nl.afpovertcp: P 
545:561(16) ack 470 win 60000 (DF)
22:15:26.875102 server.i2rs.nl.afpovertcp > apple.i2rs.nl.49156: . ack 561 
win 5840 (DF)
22:15:35.984745 server.i2rs.nl.afpovertcp > apple.i2rs.nl.49156: P 
470:486(16) ack 561 win 5840 (DF)
22:15:36.036040 apple.i2rs.nl.49156 > server.i2rs.nl.afpovertcp: . ack 486 
win 60000 (DF)
22:15:57.875009 apple.i2rs.nl.49156 > server.i2rs.nl.afpovertcp: P 
561:577(16) ack 486 win 60000 (DF)
22:15:57.875103 server.i2rs.nl.afpovertcp > apple.i2rs.nl.49156: . ack 577 
win 5840 (DF)
22:16:05.984750 server.i2rs.nl.afpovertcp > apple.i2rs.nl.49156: P 
486:502(16) ack 577 win 5840 (DF)
22:16:06.036059 apple.i2rs.nl.49156 > server.i2rs.nl.afpovertcp: . ack 502 
win 60000 (DF)
22:16:28.875017 apple.i2rs.nl.49156 > server.i2rs.nl.afpovertcp: P 
577:593(16) ack 502 win 60000 (DF)
22:16:28.875071 server.i2rs.nl.afpovertcp > apple.i2rs.nl.49156: . ack 593 
win 5840 (DF)
22:16:35.984760 server.i2rs.nl.afpovertcp > apple.i2rs.nl.49156: P 
502:518(16) ack 593 win 5840 (DF)
22:16:36.036057 apple.i2rs.nl.49156 > server.i2rs.nl.afpovertcp: . ack 518 
win 60000 (DF)
-- 

  Jeroen Baten            | EMAIL :  [email-masked]
 ____  _  __              | web   :  www.i2rs.nl
  |  )|_)(_               | tel   :  +31 (0)30 221 00 11
 _|_/_| \__)              | fax   :  +31 (0)30 220 31 91
           Kometenlaan 26, 3721 JT, Bilthoven